:100000003E292016201E2012A01A0A28A0164320DE
:10001000031831280830A9005720A80DA90B0C2877
:10002000201E3C2061205D20201A31203620280827
:1000300003103A292016201E2012201B2428FE39E6
:10004000A500201703103A29A01B2C28AC00A017EC
:100050004320031831282C084A2003183128201E79
:100060003A293C2061202013A013A012210884000B
:10007000240884178004422821088400240980056C
:10008000841780050800362061203C205D2025086B
:10009000A01A0138A8000830A900A80D03183620BE
:1000A000031C3C2061205D20A90B4D2836206120D7
:1000B0002108840024080005FF3E2208840023094B
:1000C0003F282208840023083928A8000830251971
:1000D0000130A900A80C210884002408FF3A8005FB
:1000E000841780052408031880043C30E820240885
:1000F0008004A90B6A2803143A2908302519013015
:10010000A900A801210884002408FF3A800584176B
:1001100080052408800484130005FF3E251DA80CDB
:100120002519A80D3230E820A90B842828080314CB
:100130003A29A51C3A299F28A500251C3A292108FF
:1001400084002408FF3A8005841780050130A70049
:10015000F430E920240880040130A700F430E928B5
:1001600083178001840AFF3E031DB1283A29083015
:10017000AC002518232122088400230825193221E8
:10018000251D3421210884002409841780052108B5
:100190008400A70CA60C00082404031C240680007D
:1001A000D420AC0BC7283A292208840023088006F3
:1001B000000080060800A901A800FF30A807031C62
:1001C000A907031C3A290330A700DF30E920DD2806
:1001D000A701E83EA600A709FC30031CF228A607E9
:1001E0000318EF28A6070000A70FEF282618F82805
:1001F000A61CFC280000FC280800013EAD000A30C7
:10020000A800A9010721AD0B02292A080800AB01AB
:10021000AA011030AC00270DAA0DAB0D2808AA02C8
:100220002908031C290FAB0203181D292808AA0757
:1002300029080318290FAB070310A60DA70DAC0B57
:100240000B2926083A29A801A9012A29A70CA60CDE
:10025000A80DA90DFF3E031826292908A700280884
:10026000A6003A2980043729FF3A80053829FF3A49
:10027000841780058313831203130800A00107303D
:100280009F00203084006030B120A03084005030C6
:10029000B120203084003030B020E32B0F303A05FD
:1002A000B900B908031D57290130B9009729013059
:1002B0003902031D5E290C30B9009729023039023A
:1002C000031D65290430B900972903303902031D45
:1002D0006C290930B900972904303902031D7229AD
:1002E000B901972905303902031D79290830B90071
:1002F000972906303902031D80290230B900972959
:1003000007303902031D87290B30B90097290830BF
:100310003902031D8E290A30B900972909303902A4
:10032000031D95290330B90097290F30B900390E04
:10033000F039B800F0303A05B900390E0F39B9007C
:10034000B908031DA6290130B900E6290130390298
:10035000031DAD290C30B900E62902303902031D16
:10036000B4290430B900E62903303902031DBB2942
:100370000930B900E62904303902031DC129B90149
:10038000E62905303902031DC8290830B900E629DD
:1003900006303902031DCF290230B900E6290730A3
:1003A0003902031DD6290B30B900E629083039027D
:1003B000031DDD290A30B900E62909303902031D81
:1003C000E4290330B900E6290F30B90039083807AD
:1003D000BA0008000630A1001030A4000630A200C8
:1003E0004030A3000130A5003108A600B720063038
:1003F000A600A60BF929FC290630A1001030A400A4
:100400000630A2004030A3000130A5003008A6004D
:10041000B7200630A600A60B0B2A0E2A0630A10034
:100420001030A4000630A2004030A3000130A50027
:100430002F08A600B7208316861283128616063070
:10044000A600A60B212A242A83168612831286125E
:1004500008000630A1001030A4000630A200403091
:10046000A3000130A5003208A600B7200630A60080
:10047000A60B382A3B2A0630A1001030A400063013
:10048000A2004030A3000130A5003308A600B72029
:100490000630A600A60B4A2A4D2A0630A1001030CD
:1004A000A4000630A2004030A3000130A5003408AB
:1004B000A600B72083168612831286160630A60081
:1004C000A60B602A632A83168612831286120800FE
:1004D0000630A1001030A4000630A2004030A30076
:1004E0000130A500FF30A600B7200630A600A60BFD
:1004F000772A7A2A0630A1001030A4000630A20024
:100500004030A3000130A5003508A600B720063012
:10051000A600A60B892A8C2A0630A1001030A40060
:100520000630A2004030A3000130A500FF30A60035
:10053000B72083168612831286160630A600A60BF5
:100540009F2AA22A83168612831286120800BB01F4
:1005500032303B020318322B0530A1000830A400D2
:100560000530A2000430A300D1301C2002301C2032
:100570000120B1000530A1000830A4000530A20020
:100580000430A300D1301C2001301C200120B00019
:100590000530A1000830A4000530A2000430A300FB
:1005A000D1301C2000301C200120AF00BB0A851B6D
:1005B000EF2A5930BC002F08B900BF233908AF001B
:1005C0000530A1000830A4000530A2000430A300CB
:1005D000D0301C2000301C202F081A20BB01051829
:1005E000072B5930BC003008B900BF233908B000D0
:1005F0000530A1000830A4000530A2000430A3009B
:10060000D0301C2001301C2030081A20BB01851876
:100610001F2B2430BC003108B900BF233908B100BA
:100620000530A1000830A4000530A2000430A3006A
:10063000D0301C2002301C2031081A20BB013108A8
:10064000BA004E213A08B1003008BA004E213A08EB
:10065000B0002F08BA004E213A08AF00EA219630C8
:10066000DB20A82A0800BB0132303B020318BE2B56
:100670000530A1000830A4000530A2000430A3001A
:10068000D1301C2006301C200120B4000530A10010
:100690000830A4000530A2000430A300D1301C2093
:1006A00005301C200120B3000530A1000830A40053
:1006B0000530A2000430A300D1301C2004301C20DF
:1006C0000120B200BB0A851B7B2B9930BC0034088B
:1006D000B900BF233908B4000530A1000830A400D8
:1006E0000530A2000430A300D0301C2006301C20AE
:1006F00034081A20BB010518932B1230BC003308B4
:10070000B900BF233908B3000530A1000830A400A8
:100710000530A2000430A300D0301C2005301C207E
:1007200033081A20BB018518AB2B3130BC003208CE
:10073000B900BF233908B2000530A1000830A40079
:100740000530A2000430A300D0301C2004301C204F
:1007500032081A20BB013408BA004E213A08B4000E
:100760003308BA004E213A08B3003208BA004E21CD
:100770003A08B20029229630DB20342B08000F30D3
:100780003905B800B80A0A303802031DD92BB80160
:10079000F0303905B800380E0F39B800B80A0A3001
:1007A0003802031DD52BB901D82B380EF039B9000A
:1007B000DD2BF030B9053808B90739083C020318B9
:1007C000E22BB90108000530A1001030A40001306F
:1007D000A5009C20CC306520443065200530A10068
:1007E0001030A4000130A5009C20CC306520BE3024
:1007F00065200530A1001030A4000230A5007D2046
:10080000B6007D20B70099208316061083120614C7
:10081000BD0165303D0203185B2C0530A100083096
:10082000A4000530A2000430A300D1301C20023007
:100830001C200120B1000530A1000830A4000530C3
:10084000A2000430A300D1301C2001301C20012064
:10085000B0000530A1000830A4000530A20004302B
:10086000A300D1301C2000301C200120AF0001303B
:10087000851B0301AE00013005180301AE040130F1
:1008800085180301AE040319462CA7223108BA00CB
:100890004E213A08B1003008BA004E213A08B000A3
:1008A0002F08BA004E213A08AF00EA216430DB205D
:1008B000BD0A031D092C8316061083120610831629
:1008C000861083128614BD011F303D020318B62C1A
:1008D0000530A1000830A4000530A2000430A300B8
:1008E000D1301C2006301C200120B4000530A100AE
:1008F0000830A4000530A2000430A300D1301C2031
:1009000005301C200120B3000530A1000830A400F0
:100910000530A2000430A300D1301C2004301C207C
:100920000120B2000130851B0301AE000130051823
:100930000301AE04013085180301AE040319A12C94
:1009400033233408BA004E213A08B4003308BA0001
:100950004E213A08B3003208BA004E213A08B200DC
:1009600029226430DB20BD0A031D642C8316861007
:100970008312861083168611831286150530A10016
:100980001030A4000130A5009C20CC3065204430FC
:1009900065200530A1001030A4000130A5009C2086
:1009A000CC306520BE3065200530A1001030A40099
:1009B0000230A5007D20B6007D20B7009920B70C3D
:1009C000B60CB70CB60CB70CB60CB70CB60C0F3097
:1009D000B7053608A6003708A7000130FD20BE0085
:1009E0003608A6003708A7000030FD20BF003E0EE5
:1009F000F039BE003F083E07B5003508BA004E2169
:100A00003A08B50068220B30A900B830DC20831604
:0E0A1000861183128611042C63000C2D0E2D0E
:02400E00103F61
:00000001FF
